:020000040000FA
:100000003928A000A00DA00D200D3839C1389F005F
:100010000030A100323020201F151F190D28A1012A
:100020001E083428A301A200FF30A207031CA30767
:10003000031C34280330A100DF3020201428A10144
:10004000E83EA000A109FC30031C2928A0070318E2
:100050002628A0076400A10F262820182F28A01CFE
:10006000332800003328080083130313831264002D
:100070000800831609309F000F308500860170301C
:100080008F008312860185010F30BC008611831614
:100090008611831206138316061383120130BB00E8
:1000A00064000B303B0203185C2801300120BD00C6
:1000B000C8301220BB0F5028061783160613831270
:1000C000861583168611831200300120B900013095
:1000D0000120B80002300120BA003D083C07BB00F7
:1000E000640038083B0203188A2864003B083A027F
:1000F00003187F28061383160613831264286400EE
:100100003B08390203188928861183168611831249
:100110006428922806178316061383128615831601
:0601200086118312642821
:02400E00142F6D
:00000001FF
